
 COMM

 Start     Length     Name                   Class
 0001:0000 00123H     _INIT                  CODE
 0002:0000 013CEH     _TEXT                  CODE
 0003:0000 005E5H     _INTERRUPT             CODE
 0004:0000 004D8H     _DATA                  DATA

 Origin   Group
 0004:0   DGROUP

 Address   Export                  Alias

 0002:0198 cclrbrk                 cclrbrk
 0002:0143 cevt                    cevt
 0002:015F cevtGet                 cevtGet
 0002:0107 cextfcn                 cextfcn
 0002:0123 cflush                  cflush
 0002:01D2 CommWriteString         CommWriteString
 0002:017B csetbrk                 csetbrk
 0002:00B2 ctx                     ctx
 0002:01F9 EnableNotification      EnableNotification
 0002:01B5 getdcb                  getdcb
 0002:0000 inicom                  inicom
 0002:0AC5 ReactivateOpenCommPorts  ReactivateOpenCommPorts
 0002:0073 ReadCommString          ReadCommString
 0002:004E reccom                  reccom
 0002:0019 setcom                  setcom
 0002:0032 setque                  setque
 0002:0096 sndcom                  sndcom
 0002:00E7 stacom                  stacom
 0002:0AC4 SuspendOpenCommPorts    SuspendOpenCommPorts
 0002:00CE trmcom                  trmcom
 0002:021F WEP                     WEP

  Address         Publics by Name

 0002:112F       $CLRBRK
 0002:0B67       $DCBPTR
 0002:073F       $ENANOTIFY
 0002:10AD       $EVT
 0002:10C3       $EVTGET
 0002:1173       $EXTCOM
 0002:0FE3       $FLUSH
 0002:03E3       $INICOM
 0004:0318       $MACHINEID
 0002:0D34       $RECCOM
 0002:0DF1       $RECSTR
 0002:112A       $SETBRK
 0002:0825       $SETCOM
 0002:07AF       $SETQUE
 0002:0F0B       $SNDCOM
 0002:0F5B       $SNDCOMSTR
 0002:0EDB       $SNDIMM
 0002:10DF       $STACOM
 0002:05F1       $TRMCOM
 0004:031A       ACTIVECOMS
 0000:0000  Imp  ALLOCCSTODSALIAS     (KERNEL.170)
 0003:0152       APIHANDLER
 0003:0533       CALLBACK_EVENT
 0002:0198       cclrbrk
 0002:0143       cevt
 0002:015F       cevtGet
 0002:0107       cextfcn
 0002:0123       cflush
 0002:1132       CLRBRK10
 0002:1156       CLRBRK20
 0002:1159       CLRBRK30
 0003:00BE       COMHANDLER
 0004:0000       COMM1
 0004:00A6       COMM2
 0004:014C       COMM3
 0004:01F2       COMM4
 0004:04A1       COMMBASEX
 0004:04BB       COMMDSRX
 0004:04B2       COMMFIFOX
 0003:01CE       COMMINT
 0004:04AA       COMMIRQX
 0002:01D2       CommWriteString
 0004:0298       COMPTRS
 0002:024D       CONTENTION_DLG
 0003:0006       CONTROL
 0000:0000  Imp  CreateSystemTimer    (SYSTEM.2)
 0002:017B       csetbrk
 0002:00B2       ctx
 0003:0271       DATAAVAIL
 0003:0337       DATAAVAIL100
 0003:0360       DATAAVAIL110
 0003:0370       DATAAVAIL120
 0003:0385       DATAAVAIL130
 0003:0389       DATAAVAIL140
 0003:02B4       DATAAVAIL25
 0003:02BF       DATAAVAIL30
 0003:02CE       DATAAVAIL50
 0003:02D1       DATAAVAIL60
 0003:02FB       DATAAVAIL70
 0003:0311       DATAAVAIL80
 0003:031A       DATAAVAIL90
 0002:0B75       DCBPTR10
 0003:0086       DEF_COM_INT_1
 0003:004D       DEF_COM_INT_2
 0003:0060       DEF_COM_INT_3
 0003:0073       DEF_COM_INT_4
 0003:008D       DEF_HANDLER
 0003:007D       DEF_RM_COM_INT_1
 0003:0044       DEF_RM_COM_INT_2
 0003:0057       DEF_RM_COM_INT_3
 0003:006A       DEF_RM_COM_INT_4
 0002:124C       DOLPT
 0002:1337       DOLPT40
 0002:01F9       EnableNotification
 0003:0122       ENTRY_FROM_RM
 0002:10C1       EVT10
 0002:10DD       EVTGET10
 0002:1186       EXTCOM10
 0002:118B       EXTCOM20
 0002:119C       EXTCOM30
 0002:11A1       EXTCOM40
 0002:11A8       EXTCOMDUMMY
 0002:11A4       EXTCOM_FN1
 0002:11FF       EXTCOM_FN10
 0002:11AA       EXTCOM_FN2
 0002:11B3       EXTCOM_FN3
 0002:11C0       EXTCOM_FN4
 0002:11CD       EXTCOM_FN5
 0002:11DA       EXTCOM_FN6
 0002:11E7       EXTCOM_FN7
 0002:11F1       EXTCOM_FN8
 0002:11F8       EXTCOM_FN9
 0003:01C2       FAKECOMINTFAR
 0003:03AE       FAKEXMITEMPTY
 0002:0C93       FINDCOMPORT
 0002:0FF8       FLUSH10
 0002:1009       FLUSH20
 0002:100C       FLUSH30
 0002:100F       FLUSH40
 0000:0000  Imp  FREESELECTOR         (KERNEL.176)
 0004:0336       FVPD
 0000:0000  Imp  GETAPPCOMPATFLAGS    (KERNEL.354)
 0002:02F6       GETCOMPORT386
 0002:01B5       getdcb
 0002:0B77       GETDEB
 0002:0B90       GETDEB10
 0002:0B9F       GETDEB20
 0002:0BA3       GETDEB30
 0000:0000  Imp  GETMODULEHANDLE      (KERNEL.47)
 0002:0289       GETPORT386
 0000:0000  Imp  GETPRIVATEPROFILEINT (KERNEL.127)
 0000:0000  Imp  GETPRIVATEPROFILESTRING (KERNEL.128)
 0000:0000  Imp  GETPROCADDRESS       (KERNEL.50)
 0000:0000  Imp  GETSELECTORBASE      (KERNEL.186)
 0000:0000  Imp  GetSystemMsecCount   (SYSTEM.6)
 0002:0000       inicom
 0002:0AF4       INITAPORT
 0002:042B       INITCOM10
 0002:05E7       INITCOM100
 0002:043A       INITCOM20
 0002:04B7       INITCOM40
 0002:0517       INITCOM50
 0002:058B       INITCOM59
 0002:058F       INITCOM60
 0002:05A4       INITCOM70
 0002:05C6       INITCOM80
 0002:05E2       INITCOM90
 0003:021D       INTERRUPTLOOP
 0003:0223       INTLOOP10
 0003:022E       INTLOOP20
 0004:0376       IRQHOOKS
 0002:1019       KICKTX
 0002:1032       KICKTX10
 0003:0258       LINESTAT
 0001:002A       LOADLIB
 0000:0000  Imp  LOCKSEGMENT          (KERNEL.23)
 0004:049E       LPCOMMBASE
 0004:04B8       LPCOMMDSR
 0004:04AF       LPCOMMFIFO
 0004:04A7       LPCOMMIRQ
 0004:04C5       LPCOMMSECTION
 0004:0320       LPFNMESSAGEBOX
 0004:0324       LPFNVPD
 0004:031C       LPPOSTMESSAGE
 0004:04CC       LPSYSTEMINI
 0004:02A0       LPT1
 0004:02C8       LPT2
 0004:02F0       LPT3
 0002:1310       LPT_GETSTATUS
 0002:128C       LPT_OUTCHAR
 0002:125C       LPT_RESET
 0002:12E6       LPT_STROBE
 0003:04A9       MODEMSTATUS
 0003:04E8       MODEMSTATUS10
 0003:04FF       MODEMSTATUS20
 0003:04F9       MODEMSTATUS30
 0002:1049       MSRRESTART
 0002:1048       MSRWAIT
 0002:104B       MSRWAIT10
 0002:104E       MSRWAIT20
 0002:1069       MSRWAIT30
 0002:1077       MSRWAIT40
 0002:1083       MSRWAIT50
 0002:1092       MSRWAIT60
 0002:109F       MSRWAIT70
 0002:10A2       MSRWAIT80
 0002:10A9       MSRWAIT90
 0003:050B       NOTIFY_OWNER
 0003:039D       OUTHANDSHAKINGCHAR
 0004:042D       PCOMBYTE
 0004:03C5       PLPTBYTE
 0002:0AC5       ReactivateOpenCommPorts
 0002:0073       ReadCommString
 0002:004E       reccom
 0002:0DEC       RECCOM100
 0002:0D83       RECCOM40
 0002:0D9B       RECCOM50
 0002:0DA7       RECCOM60
 0002:0DC4       RECCOM70
 0002:0DD6       RECCOM80
 0002:0DDB       RECCOM90
 0002:0DEA       RECCOM95
 0003:0147       RM_APIHANDLER
 0003:0002       RM_CALLBACK
 0003:0000       RM_INTDATASEG
 0002:0CFD       ROTATE_PIC
 0002:0226       SEGMENTFROMSELECTOR
 0002:0F14       SENDCOM10
 0002:0F1B       SENDCOM20
 0002:0F3A       SENDCOM30
 0002:0F4F       SENDCOM40
 0002:0F52       SENDCOM50
 0002:0F56       SENDCOM60
 0002:0EF1       SENDIMM10
 0002:0F09       SENDIMM20
 0002:0019       setcom
 0002:083A       SETCOM10
 0002:083F       SETCOM20
 0002:09F7       SETCOM210
 0002:09FF       SETCOM220
 0002:0A07       SETCOM230
 0002:0A0F       SETCOM240
 0002:0A4A       SETCOM310
 0002:0A7C       SETCOM410
 0002:0A80       SETCOM420
 0002:0A8A       SETCOM430
 0002:0AA9       SETCOM440
 0002:0AAB       SETCOM450
 0002:0ABA       SETCOM460
 0002:0ABF       SETCOM470
 0002:0838       SETCOM5
 0002:0032       setque
 0002:0822       SETQUE10
 0002:0096       sndcom
 0002:00E7       stacom
 0002:1118       STACOM20
 0002:1123       STACOM25
 0002:1128       STACOM30
 0002:038B       STEALPORT
 0002:1366       STRINGTOLPT
 0002:0AC4       SuspendOpenCommPorts
 0004:0426       SZCOMMESSAGE
 0004:03BE       SZMESSAGE
 0002:0610       TERMCOM10
 0002:061C       TERMCOM15
 0002:0630       TERMCOM20
 0002:0631       TERMCOM30
 0002:0639       TERMCOM60
 0002:063C       TERMINATE
 0002:0646       TERMINATE10
 0002:0654       TERMINATE20
 0002:065B       TERMINATE30
 0002:06A9       TERMINATE45
 0002:070E       TERMINATE49
 0002:0640       TERMINATE5
 0002:073C       TERMINATE50
 0003:0556       TIMERPROC
 0002:00CE       trmcom
 0002:1012       TXI
 0000:0000  Imp  UNLOCKSEGMENT        (KERNEL.24)
 0004:0319       USING_DPMI
 0004:0330       VCD_INT_CALLBACK
 0002:021F       WEP
 0000:0000  Imp  WOWCLOSECOMPORT      (KERNEL.509)
 0003:03D1       XMITEMPTY
 0003:03E4       XMITEMPTY10
 0003:04A1       XMITEMPTY100
 0003:04A5       XMITEMPTY110
 0003:03EF       XMITEMPTY20
 0003:03F5       XMITEMPTY30
 0003:03FE       XMITEMPTY40
 0003:0460       XMITEMPTY59
 0003:0477       XMITEMPTY60
 0003:049D       XMITEMPTY90
 0004:048E       _SZTITLE
 0000:0000  Imp  __0040H              (KERNEL.193)
 0000:0000  Imp  __F000H              (KERNEL.194)
 0000:0000  Imp  __WINFLAGS           (KERNEL.178)

  Address         Publics by Value

 0000:0000  Imp  GETPRIVATEPROFILESTRING (KERNEL.128)
 0000:0000  Imp  GETPRIVATEPROFILEINT (KERNEL.127)
 0000:0000  Imp  ALLOCCSTODSALIAS     (KERNEL.170)
 0000:0000  Imp  WOWCLOSECOMPORT      (KERNEL.509)
 0000:0000  Imp  GetSystemMsecCount   (SYSTEM.6)
 0000:0000  Imp  CreateSystemTimer    (SYSTEM.2)
 0000:0000  Imp  UNLOCKSEGMENT        (KERNEL.24)
 0000:0000  Imp  __WINFLAGS           (KERNEL.178)
 0000:0000  Imp  __F000H              (KERNEL.194)
 0000:0000  Imp  LOCKSEGMENT          (KERNEL.23)
 0000:0000  Imp  GETPROCADDRESS       (KERNEL.50)
 0000:0000  Imp  GETAPPCOMPATFLAGS    (KERNEL.354)
 0000:0000  Imp  FREESELECTOR         (KERNEL.176)
 0000:0000  Imp  GETSELECTORBASE      (KERNEL.186)
 0000:0000  Imp  __0040H              (KERNEL.193)
 0000:0000  Imp  GETMODULEHANDLE      (KERNEL.47)
 0001:002A       LOADLIB
 0002:0000       inicom
 0002:0019       setcom
 0002:0032       setque
 0002:004E       reccom
 0002:0073       ReadCommString
 0002:0096       sndcom
 0002:00B2       ctx
 0002:00CE       trmcom
 0002:00E7       stacom
 0002:0107       cextfcn
 0002:0123       cflush
 0002:0143       cevt
 0002:015F       cevtGet
 0002:017B       csetbrk
 0002:0198       cclrbrk
 0002:01B5       getdcb
 0002:01D2       CommWriteString
 0002:01F9       EnableNotification
 0002:021F       WEP
 0002:0226       SEGMENTFROMSELECTOR
 0002:024D       CONTENTION_DLG
 0002:0289       GETPORT386
 0002:02F6       GETCOMPORT386
 0002:038B       STEALPORT
 0002:03E3       $INICOM
 0002:042B       INITCOM10
 0002:043A       INITCOM20
 0002:04B7       INITCOM40
 0002:0517       INITCOM50
 0002:058B       INITCOM59
 0002:058F       INITCOM60
 0002:05A4       INITCOM70
 0002:05C6       INITCOM80
 0002:05E2       INITCOM90
 0002:05E7       INITCOM100
 0002:05F1       $TRMCOM
 0002:0610       TERMCOM10
 0002:061C       TERMCOM15
 0002:0630       TERMCOM20
 0002:0631       TERMCOM30
 0002:0639       TERMCOM60
 0002:063C       TERMINATE
 0002:0640       TERMINATE5
 0002:0646       TERMINATE10
 0002:0654       TERMINATE20
 0002:065B       TERMINATE30
 0002:06A9       TERMINATE45
 0002:070E       TERMINATE49
 0002:073C       TERMINATE50
 0002:073F       $ENANOTIFY
 0002:07AF       $SETQUE
 0002:0822       SETQUE10
 0002:0825       $SETCOM
 0002:0838       SETCOM5
 0002:083A       SETCOM10
 0002:083F       SETCOM20
 0002:09F7       SETCOM210
 0002:09FF       SETCOM220
 0002:0A07       SETCOM230
 0002:0A0F       SETCOM240
 0002:0A4A       SETCOM310
 0002:0A7C       SETCOM410
 0002:0A80       SETCOM420
 0002:0A8A       SETCOM430
 0002:0AA9       SETCOM440
 0002:0AAB       SETCOM450
 0002:0ABA       SETCOM460
 0002:0ABF       SETCOM470
 0002:0AC4       SuspendOpenCommPorts
 0002:0AC5       ReactivateOpenCommPorts
 0002:0AF4       INITAPORT
 0002:0B67       $DCBPTR
 0002:0B75       DCBPTR10
 0002:0B77       GETDEB
 0002:0B90       GETDEB10
 0002:0B9F       GETDEB20
 0002:0BA3       GETDEB30
 0002:0C93       FINDCOMPORT
 0002:0CFD       ROTATE_PIC
 0002:0D34       $RECCOM
 0002:0D83       RECCOM40
 0002:0D9B       RECCOM50
 0002:0DA7       RECCOM60
 0002:0DC4       RECCOM70
 0002:0DD6       RECCOM80
 0002:0DDB       RECCOM90
 0002:0DEA       RECCOM95
 0002:0DEC       RECCOM100
 0002:0DF1       $RECSTR
 0002:0EDB       $SNDIMM
 0002:0EF1       SENDIMM10
 0002:0F09       SENDIMM20
 0002:0F0B       $SNDCOM
 0002:0F14       SENDCOM10
 0002:0F1B       SENDCOM20
 0002:0F3A       SENDCOM30
 0002:0F4F       SENDCOM40
 0002:0F52       SENDCOM50
 0002:0F56       SENDCOM60
 0002:0F5B       $SNDCOMSTR
 0002:0FE3       $FLUSH
 0002:0FF8       FLUSH10
 0002:1009       FLUSH20
 0002:100C       FLUSH30
 0002:100F       FLUSH40
 0002:1012       TXI
 0002:1019       KICKTX
 0002:1032       KICKTX10
 0002:1048       MSRWAIT
 0002:1049       MSRRESTART
 0002:104B       MSRWAIT10
 0002:104E       MSRWAIT20
 0002:1069       MSRWAIT30
 0002:1077       MSRWAIT40
 0002:1083       MSRWAIT50
 0002:1092       MSRWAIT60
 0002:109F       MSRWAIT70
 0002:10A2       MSRWAIT80
 0002:10A9       MSRWAIT90
 0002:10AD       $EVT
 0002:10C1       EVT10
 0002:10C3       $EVTGET
 0002:10DD       EVTGET10
 0002:10DF       $STACOM
 0002:1118       STACOM20
 0002:1123       STACOM25
 0002:1128       STACOM30
 0002:112A       $SETBRK
 0002:112F       $CLRBRK
 0002:1132       CLRBRK10
 0002:1156       CLRBRK20
 0002:1159       CLRBRK30
 0002:1173       $EXTCOM
 0002:1186       EXTCOM10
 0002:118B       EXTCOM20
 0002:119C       EXTCOM30
 0002:11A1       EXTCOM40
 0002:11A4       EXTCOM_FN1
 0002:11A8       EXTCOMDUMMY
 0002:11AA       EXTCOM_FN2
 0002:11B3       EXTCOM_FN3
 0002:11C0       EXTCOM_FN4
 0002:11CD       EXTCOM_FN5
 0002:11DA       EXTCOM_FN6
 0002:11E7       EXTCOM_FN7
 0002:11F1       EXTCOM_FN8
 0002:11F8       EXTCOM_FN9
 0002:11FF       EXTCOM_FN10
 0002:124C       DOLPT
 0002:125C       LPT_RESET
 0002:128C       LPT_OUTCHAR
 0002:12E6       LPT_STROBE
 0002:1310       LPT_GETSTATUS
 0002:1337       DOLPT40
 0002:1366       STRINGTOLPT
 0003:0000       RM_INTDATASEG
 0003:0002       RM_CALLBACK
 0003:0006       CONTROL
 0003:0044       DEF_RM_COM_INT_2
 0003:004D       DEF_COM_INT_2
 0003:0057       DEF_RM_COM_INT_3
 0003:0060       DEF_COM_INT_3
 0003:006A       DEF_RM_COM_INT_4
 0003:0073       DEF_COM_INT_4
 0003:007D       DEF_RM_COM_INT_1
 0003:0086       DEF_COM_INT_1
 0003:008D       DEF_HANDLER
 0003:00BE       COMHANDLER
 0003:0122       ENTRY_FROM_RM
 0003:0147       RM_APIHANDLER
 0003:0152       APIHANDLER
 0003:01C2       FAKECOMINTFAR
 0003:01CE       COMMINT
 0003:021D       INTERRUPTLOOP
 0003:0223       INTLOOP10
 0003:022E       INTLOOP20
 0003:0258       LINESTAT
 0003:0271       DATAAVAIL
 0003:02B4       DATAAVAIL25
 0003:02BF       DATAAVAIL30
 0003:02CE       DATAAVAIL50
 0003:02D1       DATAAVAIL60
 0003:02FB       DATAAVAIL70
 0003:0311       DATAAVAIL80
 0003:031A       DATAAVAIL90
 0003:0337       DATAAVAIL100
 0003:0360       DATAAVAIL110
 0003:0370       DATAAVAIL120
 0003:0385       DATAAVAIL130
 0003:0389       DATAAVAIL140
 0003:039D       OUTHANDSHAKINGCHAR
 0003:03AE       FAKEXMITEMPTY
 0003:03D1       XMITEMPTY
 0003:03E4       XMITEMPTY10
 0003:03EF       XMITEMPTY20
 0003:03F5       XMITEMPTY30
 0003:03FE       XMITEMPTY40
 0003:0460       XMITEMPTY59
 0003:0477       XMITEMPTY60
 0003:049D       XMITEMPTY90
 0003:04A1       XMITEMPTY100
 0003:04A5       XMITEMPTY110
 0003:04A9       MODEMSTATUS
 0003:04E8       MODEMSTATUS10
 0003:04F9       MODEMSTATUS30
 0003:04FF       MODEMSTATUS20
 0003:050B       NOTIFY_OWNER
 0003:0533       CALLBACK_EVENT
 0003:0556       TIMERPROC
 0004:0000       COMM1
 0004:00A6       COMM2
 0004:014C       COMM3
 0004:01F2       COMM4
 0004:0298       COMPTRS
 0004:02A0       LPT1
 0004:02C8       LPT2
 0004:02F0       LPT3
 0004:0318       $MACHINEID
 0004:0319       USING_DPMI
 0004:031A       ACTIVECOMS
 0004:031C       LPPOSTMESSAGE
 0004:0320       LPFNMESSAGEBOX
 0004:0324       LPFNVPD
 0004:0330       VCD_INT_CALLBACK
 0004:0336       FVPD
 0004:0376       IRQHOOKS
 0004:03BE       SZMESSAGE
 0004:03C5       PLPTBYTE
 0004:0426       SZCOMMESSAGE
 0004:042D       PCOMBYTE
 0004:048E       _SZTITLE
 0004:049E       LPCOMMBASE
 0004:04A1       COMMBASEX
 0004:04A7       LPCOMMIRQ
 0004:04AA       COMMIRQX
 0004:04AF       LPCOMMFIFO
 0004:04B2       COMMFIFOX
 0004:04B8       LPCOMMDSR
 0004:04BB       COMMDSRX
 0004:04C5       LPCOMMSECTION
 0004:04CC       LPSYSTEMINI

Program entry point at 0001:002a
